:0A1F2B00000102020303040405058F
:10060100E4F513F512F511F510C203C200C202C2DE
:1006110001121E55120AB37E167F008E518F52753C
:100621005916755A12754F1675501C75571675580F
:100631004A755B16755C78EE54E0700302074875E5
:1006410014007515808E168F17C374A29FFF741640
:100651009ECF2402CF3400FEE48F0F8E0EF50DF5F0
:100661000CF50BF50AF509F508AF0FAE0EAD0DACA3
:100671000CAB0BAA0AA909A808C312092C5026E53C
:1006810015250BF582E514350AF58374CDF0E50BDC
:100691002401F50BE4350AF50AE43509F509E435D9
:1006A10008F50880C4E4F50BF50AF509F508AF0F64
:1006B100AE0EAD0DAC0CAB0BAA0AA909A808C3126A
:1006C100092C5031AE0AAF0BE5172FF582E5163E26
:1006D100F583E0FDE5152FF582E5143EF583EDF098
:1006E100EF2401F50BE43EF50AE43509F509E4359B
:1006F10008F50880B985145185155274002480FFCE
:10070100741634FFFEC3E55A9FF55AE5599EF55913
:10071100C3E5549FF554E5539EF553C3E5569FF544
:1007210056E5559EF555C3E5509FF550E54F9EF5AD
:100731004FC3E5589FF558E5579EF557C3E55C9FB4
:10074100F55CE55B9EF55BD2E843D82090E668E076
:100751004409F090E65CE0443DF0D2AF90E680E0E1
:1007610020E105D208121C9090E680E054F7F05386
:100771008EF8C2033001051203DDC20130032912D4
:1007810011FE5024C203121E1420001690E682E0CE
:1007910030E704E020E1EF90E682E030E604E0207B
:0D07A100E0E4121D1912201C12173F80C742
:1003DD0090E6B9E0700302048E14700302050B243D
:1003ED00FE700302058E24FB700302048814700353
:1003FD00020482146073146076240560030205ED17
:10040D0012201E40030205F990E6BBE024FE602297
:10041D0014603324FD601114602224067048E551E8
:10042D0090E6B3F0E5528037E55990E6B3F0E55A22
:10043D00802DE55390E6B3F0E5548023E55590E625
:10044D00B3F0E556801990E6BAE0FF121D45AA06F5
:10045D00A9077B01EA494B600DEE90E6B3F0EF90F2
:10046D00E6B4F00205F90205F2121EF30205F912C7
:10047D001F9C0205F9121AA30205F9121EE10205CD
:10048D00F912202040030205F990E6B8E0247F60C0
:10049D001514601924027063A200E43325E0FFA255
:1004AD0002E4334F8041E490E740F0803F90E6BC9A
:1004BD00E0547EFF7E00E0D394807C0040047D01FB
:1004CD0080027D00EC4EFEED4F242BF582741F3E15
:1004DD00F583E493FF3395E0FEEF24A1FFEE34E6C0
:1004ED008F82F583E0540190E740F0E4A3F090E6AD
:1004FD008AF090E68B7402F00205F90205F21220E3
:10050D002240030205F990E6B8E024FE60162402AD
:10051D0060030205F990E6BAE0B40105C2000205D8
:10052D00F90205F290E6BAE0705590E6BCE0547E13
:10053D00FF7E00E0D394807C0040047D0180027D2D
:10054D0000EC4EFEED4F242BF582741F3EF583E437
:10055D0093FF3395E0FEEF24A1FFEE34E68F82F595
:10056D0083E054FEF090E6BCE05480131313541F47
:10057D00FFE0540F2F90E683F0E04420F0806D8073
:10058D0064122024506690E6B8E024FE601924021F
:10059D00705A90E6BAE0B40104D200804F90E6BAEA
:1005AD00E064026047803E90E6BCE0547EFF7E0032
:1005BD00E0D394807C0040047D0180027D00EC4EF0
:1005CD00FEED4F242BF582741F3EF583E493FF332C
:1005DD0095E0FEEF24A1FFEE34E68F82F5838008CF
:1005ED00120080500790E6A0E04401F090E6A0E0F4
:0305FD004480F047
:0106000022D7
:03003300022008A0
:0420080053D8EF3288
:101E5500758CE0758AC0E58954F04401F589758E65
:081E650003D28CD2A9D2AF22F6
:03000B000214C418
:1014C400C0E0C0F0C083C082C0D075D000C000C0EE
:1014D40001C002C003C004C005C006C007758CE08B
:1014E400758AC0D28CE47F607EEAFDFCAB4EAA4DC7
:1014F400A94CA84BC312092C5019AF4EAE4DAD4C9C
:10150400AC4BEF2401F54EE43EF54DE43DF54CE4DF
:101514003CF54BE47F01FEFDFCAB4EAA4DA94CA863
:101524004BC312092C7008E5A054F02534F5A0E54E
:101534002B2401FFE4352AFEE4FCFDAB4EAA4DA9A1
:101544004CA84BC312092C700553A0F0C28CD007D1
:10155400D006D005D004D003D002D001D000D0D022
:09156400D082D083D0F0D0E03237
:1016000012010002000000401816056000000102EF
:1016100000010A06000200000040010009022E003D
:1016200001010080FA0904000004FF000000070522
:1016300001024000000705820200020007050202C5
:101640000002000705810240000009022E0001018E
:101650000080FA0904000004FF00000007050102F1
:101660004000000705820240000007050202000258
:101670000007058102400000040309041003510023
:10168000480059002D004300430044001603510058
:10169000480059002D0038004C0020002000200098
:0416A0002000000026
:100FF00060802800010402020202020700000002D1
:10100000000002001332120A080C08000000000061
:101010000000003F01040202020202070000000279
:101020000000020013320A12100C08000000000039
:101030000000003F031A030303030307000000023C
:10104000000002001332120A080C08000000000021
:101050000000003F035A03030303030700000002DC
:101060000000020013320A12100C080000000000F9
:101070000000003F602428870000000000000000FE
:101080000000000000000000000000000000000060
:1010900000000000000000000000000047288080E1
:0610A000000000CA4E0032
:1010B90090E60174CAF090E6F574FFF0902880E09C
:1010C90090E6F3F0902881E090E6C3F0902882E062
:1010D90090E6C1F0902883E090E6C2F0902885E080
:1010E90090E6C0F0902886E090E6F4F075AF0774BA
:1010F90028F59A7400F59B759DE4E4F59EFF90E64A
:101109007BE090E67CF00FBF80F490E67174FFF00D
:10111900F5B490E672E04480F043B680000000E444
:1011290090E6C4F000000090E6C5F0902887E090B2
:10113900E6C6F0902888E090E6C7F0902889E0900C
:10114900E6C8F090288AE090E6C9F090288BE090F4
:10115900E6CAF090288CE090E6CBF090288DE090DC
:0B116900E6CCF090288EE090E6CDF080
:011174002258
:03004300021200A6
:0300530002120096
:10120000021E6D00021ECB00021EB500021E8500EC
:10121000021B8C00021AE000022026000220270098
:101220000220280002202900021979000216A400D9
:1012300002202A0002202B0002202C0002202D0078
:1012400002202E000220270002202F000220300062
:10125000022031000220320002203300022034003C
:10126000022035000220270002202700022027004C
:101270000220360002203700022038000220390008
:1012800002203A0002203B0002203C0002203D00E8
:1012900002203E0002203F000220400002204100C8
:1012A00002204200022043000220440002204500A8
:0812B000022046000220470065
:101D190090E682E030E004E020E60B90E682E030D5
:101D2900E119E030E71590E680E04401F07F147E88
:0C1D390000121A1E90E680E054FEF0221A
:101E140090E682E044C0F090E681F0438701000040
:041E24000000002298
:101C900030080990E680E0440AF0800790E680E092
:101CA0004408F07FDC7E05121A1E90E65D74FFF09A
:0F1CB00090E65FF05391EF90E680E054F7F0225A
:021D4500A907EC
:101D4700AE5BAF5C8F828E83A3E064037017AD0137
:101D570019ED7001228F828E83E07C002FFDEC3E0F
:091D6700FEAF0580DF7E007F0065
:011D70002250
:101A1E008E1E8F1F90E600E054187012E51F2401F1
:101A2E00FFE4351EC313F51EEF13F51F801590E668
:101A3E0000E05418FFBF100BE51F25E0F51FE51E53
:101A4E0033F51EE51F151FAE1E7002151E4E6005E6
:061A5E00121E2880EE229A
:101E28007400F58690FDA57C05A3E582458370F9CD
:011E38002287
:1010A600C1850223000002311040C1070447000039
:0210B600000038
:081D710090E679F07F057E0089
:101D79008E1E8F1FE51F451E60177F957E00121A64
:101D890007000000000000E51F151F70E7151E8001
:021D9900E32243
:100AB30090E600E054E74410F000000000000090CE
:100AC300E61074A0F000000090E60B7401F090E6CD
:100AD3001274E0F0000000E490E613F000000090D0
:100AE300E614F000000090E615F000000090E61810
:100AF300740CF000000090E6D27402F090E60474E7
:100B030080F00000007402F0000000E4F000000038
:100B13001210B9E490E671F075B4FF90E672F075C7
:100B2300B6FF75B1FF90E670F075B2FFC28CD28745
:100B3300D285121F1475230275240000000090E66D
:100B43001074A0F000000000000090E611F0000017
:100B53000090E65EE04408F0000000E490E68DF0CB
:100B630090E65EE04404F0000000E490E68FF012AB
:100B73001CBF5380FE7F9A7E00121F5D752800758F
:100B830029B47542017543907531107532B87545B6
:100B93000675462C121FAC90E67AE054FEF0E4FD95
:100BA3007F90121C2C7F647E00121A1E7DFF7F42F1
:100BB300121C2C7F647E00121A1E7D827F4E121C33
:100BC3002C7535FF75388290E782E535F090E78123
:090BD300E538F01215FB021F14B5
:10117500E538D3940040037535FF90E678E0448068
:10118500F07491121D7190E679E090E7C0121D741C
:1011950090E679E090E7C1121D7490E679E090E75A
:1011A500C2121D7490E679E090E7C3121D7490E6B3
:1011B50078E04440121D7490E678E04480F0744273
:1011C500121D7190E679E535121D7490E678E044BC
:1011D50040121D7490E678E04480F090E679744EF4
:1011E500121D7490E679E538121D7490E678E04496
:0911F50040F07F057E00021D7927
:10173F00E54A2401F54AE43549F549E43548F548C9
:10174F00E43547F547E47FE87E03FDFCAB4AAA4941
:10175F00A948A847C312092C7006FD7F90121C2CB4
:10176F007FA07E867D017C00AB4AAA49A948A84785
:10177F00C312092C7009121F261211751215FB7F47
:10178F00407E0D7D037C00AB4AAA49A948A847D3E8
:10179F0012092C4009E4F54AF549F548F54730049C
:1017AF0020E533B4010312136AE533B402031218B0
:1017BF0060E533B4040312156DE533B46303120906
:0417CF003DC20422F1
:0211FE00D322FA
:02201C00D322CD
:02201E00D322CB
:101AA30090E680E030E71800000090E6207402F032
:101AB300000000E490E621F0000000D2058016004B
:101AC3000000E490E620F000000090E6217440F06E
:0D1AD300000000C20590E6BAE0F540D32205
:101EE10090E740E540F0E490E68AF090E68B04F05C
:021EF100D322FA
:081F9C0090E6BAE0F527D3221C
:101EF30090E740E527F0E490E68AF090E68B04F063
:021F0300D322E7
:02202000D322C9
:02202200D322C7
:02202400D322C5
:10008000E4F518F51990E6B9E0244B606B147003A1
:1000900002023C24F4700302027424FD7003020285
:1000A000BF14700302032324FD70030203582416B7
:1000B00060030203D9E490E68AF090E68BF090E6C4
:1000C000A0E020E1F990E68BE0F518E4F5B5F5B392
:1000D00090E60174CAF0E490E6C3F090E6C2F0D274
:1000E0000400000090E6047480F00000007402F048
:1000F000000000E4F00203DBE490E68AF090E68B77
:10010000F090E6A0E020E1F990E68BE0F518D394BA
:100110003F4024E4F51974402519F582E434E7F5ED
:1001200083E0FF74AB2519F582E43428F583EFF002
:100130000519E519B440DF7F9A7E00121F5D9028F3
:10014000ABE0FF7E00121F669028ABE0FF7E00123E
:100150001F6F9028ABE0FF7E00121F789028ACE064
:1001600075F004A4FFAEF0121F819028ACE075F08A
:1001700004A4FFAEF0121F8A9028ACE075F004A42E
:10018000FFAEF0121F939028B0E0C394025013907A
:1001900028CCE090E6C07005744EF08016749CF098
:1001A00080119028CCE090E6C07005749FF0800329
:1001B000749DF09028CEE0F5399028CBE0F537908B
:1001C00028DAE0FEA3E07C002400F526EC3EF525CD
:1001D0009028B1E0F533E53370037533019028B60C
:1001E000E0FEA3E07C002400F529EC3EF528A3E026
:1001F000FEA3E02400F543EC3EF5429028B2E0FE79
:10020000A3E02400F532EC3EF531A3E0FEA3E024A8
:1002100000F546EC3EF5459028BCE0FEA3E0240046
:10022000F53FEC3EF53E9028BAE0FEA3E02400F551
:1002300030EC3EF52FE4FD7F90020352E4F5197493
:10024000AB2519F582E43428F583E0FF74402519C5
:10025000F582E434E7F583EFF00519E519B40ADF18
:10026000000000E490E68AF000000090E68B740A3B
:10027000F00203DB90E74074B2F0A37411F0A374B2
:100280000CF0A37426F0A37407F0A374EEF0A3742B
:1002900001F0A37403F0A37413F0300505E4A3F098
:1002A000800690E74974FFF0000000E490E68AF0D1
:1002B00000000090E68B740AF0121CBF0203DB9072
:1002C000E678E04480F090E6797491F07F647E00F7
:1002D000121A0790E679E090E740F07F647E001202
:1002E0001A0790E679E090E741F07F647E00121AE9
:1002F0000790E679E090E742F07F647E00121A07EB
:1003000090E679E090E743F090E678E04440F00032
:100310000000E490E68AF000000090E68B7404F0A0
:100320000203DBE490E68AF090E68BF090E6A0E032
:1003300020E1F990E68BE0F518D394015003020315
:10034000DB90E741E0FD7F42121C2C90E740E0FD8E
:100350007F4E121C2C0203DBE490E68AF090E68BC1
:10036000F090E6A0E020E1F990E68BE0F518D39458
:1003700001406890E740E05480C4131313540124F3
:10038000FF92A3E05440C41313540324FF92A2E04D
:100390005420C413540724FF92A1E05410C4540FF6
:1003A00024FF92A0A3E075F00AA4FFAEF0121A1E7B
:1003B00090E740E05408131313541F24FF92A3E066
:1003C00054041313543F24FF92A2E05402C3132495
:0C03D000FF92A1E01392A08002D322C390
:0103DC0022FE
:101E6D00C0E0C083C082D2015391EF90E65D740152
:081E7D00F0D082D083D0E032E6
:101EB500C0E0C083C0825391EF90E65D7404F0D01A
:061EC50082D083D0E03260
:101ECB00C0E0C083C0825391EF90E65D7402F0D006
:061EDB0082D083D0E0324A
:101B8C00C0E0C083C08285575385585485548285E4
:101B9C005383A37402F0854F558550568556828524
:101BAC005583A37407F05391EF90E65D7410F0D059
:061BBC0082D083D0E0326C
:101E8500C0E0C083C082D2035391EF90E65D740831
:081E9500F0D082D083D0E032CE
:101AE000C0E0C083C08290E680E030E720854F539D
:101AF000855054855482855383A37402F0855755CD
:101B0000855856855682855583A37407F05391EF07
:0D1B100090E65D7420F0D082D083D0E032EA
:012026003287
:012027003286
:012028003285
:012029003284
:10197900C0E0C0F0C083C082C0D075D000C000C034
:1019890001C002C003C004C005C006C007C2AF122F
:101999001F2600000090E68F7404F00000005391A8
:1019A900EF90E65FE04404F01215FBD2AFD007D008
:1019B90006D005D004D003D002D001D000D0D0D0B9
:0819C90082D083D0F0D0E0329F
:1016A400C0E0C083C082C0D075D000C004C006C0F2
:0116B400072E
:1016B500C2AF90E6A1E020E1F990E780E014601464
:1016C50024F8601E240C604624FE6046147048759C
:1016D5002200804390E782E0F53590E781E0F53818
:1016E5008035D28C90E781E0540FF534A3E0FEA35A
:1016F500E07C002400FFEC3EC313F52AEF13F52B25
:10170500754E00754D00754C00754B008009C28CF7
:101715008005752200D20600000090E68DE4F053A6
:0B17250091EF90E65FE04408F0D2AFC7
:0F173000D007D006D004D0D0D082D083D0E03202
:01202A003283
:01202B003282
:01202C003281
:01202D003280
:01202E00327F
:01202F00327E
:01203000327D
:01203100327C
:01203200327B
:01203300327A
:012034003279
:012035003278
:012036003277
:012037003276
:012038003275
:012039003274
:01203A003273
:01203B003272
:01203C003271
:01203D003270
:01203E00326F
:01203F00326E
:01204000326D
:01204100326C
:01204200326B
:01204300326A
:012044003269
:012045003268
:012046003267
:012047003266
:060F26008F1A8C1B8D1CCC
:100F2C00531A0753A0BF7F0A7E00121A07E4F51D5F
:100F3C00F51EC37402951EFFE51AA807088002C3AC
:100F4C0013D8FC30E00543A020800353A0DF7F0AB8
:100F5C007E00121A0743A0107F0A7E00121A075354
:100F6C00A0EF7F0A7E00121A07051EE51E7002050F
:100F7C001DC39403E51D6480948040B6E4F51DF513
:100F8C001EC37409951EFFE51CAE1BA8070880053F
:100F9C00CEC313CE13D8F930E00543A02080035301
:100FAC00A0DF7F0A7E00121A0743A0107F0A7E0082
:100FBC00121A0753A0EF7F0A7E00121A07051EE5CE
:100FCC001E7002051DC3940AE51D6480948040B117
:100FDC0043A0407F0A7E00121A0753A0BF7F0A7EEF
:040FEC0000021A07DE
:091F5D00AD07AC06E4FF020F26FB
:091F6600AD07AC067F04020F2652
:091F6F00AD07AC067F05020F2648
:091F7800AD07AC067F06020F263E
:091F8100AD07AC067F01020F263A
:091F8A00AD07AC067F02020F2630
:091F9300AD07AC067F03020F2626
:101C2C008D1AAD0790E678E04480F090E679EDF0FF
:101C3C007F647E00121A0790E679E51AF07F647EC5
:101C4C0000121A0790E678E04440F07F647E0002B0
:021C5C001A0765
:1019D1007F147E00121A071220147F037E00121A50
:1019E100071220107F027E00121A07121F497F0280
:1019F1007E00121A07121F537F027E00121A07126D
:061A0100200C7F027E00B4
:101A0700EF7803C333CE33CED8F9FFEF4E6007EF3D
:071A17001F70F81E80F5228C
:071FB40053B1EF53B1BF224E
:071FBB0053B1EF43B14022D6
:071FC20043B11043B14022BE
:071FC90053B1FE53B1FB22EE
:071FD00053B1FE43B10422EE
:071FD70043B10143B10422F4
:04200C0053B1F722B3
:0420100043B10822AE
:0420140053B17F2223
:0420180043B180222E
:071FDE0053B1EF53B1DF2204
:071FE50053B1EF43B12022CC
:071FEC0043B11043B12022B4
:071FF30053B1FE53B1FD22C2
:071FFA0053B1FE43B10222C6
:0720010043B10143B10222CB
:0A1F350053B1EF53B1BF53B1DF22E7
:0A1F3F0053B1FE53B1FB53B1FD2274
:0A1F490053B1EF43B14043B1202231
:051F05007E00121A0726
:0A1F0A0053B1FE43B10443B10222BB
:101A6400E4FFFEE53BFDE4FCFB7A01F9F812089A79
:101A7400E4FB7A01F9F812089A8F2CE4FFE53CFEA6
:101A8400E4FDFCFB7A01F9F812089A8F2EE53DFF7C
:051A94008F2D1220104F
:0A1A990043B11043B14043B12022D5
:0A1F530043B10143B10443B102227F
:0C1F1400121F4912200C121F530220184B
:101D9B00121F147F0A7E00121A07121F357F037E53
:101DAB0000121A07121F49121F0A121A991219D17F
:0A1DBB001220187F147E00021A07A0
:101DED00121F147F0A121F057F037E00121A07129D
:101DFD001A99121F3F7F08121F051219D1122018B0
:071E0D007F147E00021A079A
:031E3900121DC5B2
:101E3C007F01121F05121A03121A99121A0312208B
:091E4C00147F021219DD022018B6
:101E9D00121F14121A03E4FDFC121E3C0DBD0001AD
:071EAD000CBC03F5BDF7F2C8
:011EB400220B
:081FA400C285121A03D2852246
:101CBF00C283E4F51AF51BD2827F1E7E00121A1E14
:101CCF00C2827F1E7E00121A1E051BE51B700205C5
:0C1CDF001AC39405E51A6480948040DB71
:011CEB0022D6
:061F2000121DED121D9BD5
:051F2600C283C282220B
:0515FB00D283D2822220
:012048002275
:012049002274
:1017D300121A64E530452F7003121FA4E537B401D4
:1017E30002C287122048E539706AE52C75F040A4DF
:1017F30085F01CF51DAF227E00AC1CAD1D1207FD4C
:10180300D3EF9400EE940040147FC47E03121D793D
:10181300121175E51D151D70DC151C80D8751C0093
:10182300852E1DAF227E00AC1CAD1D1207FDD3EF2C
:101833009400EE940040147FC47E00121D791211AF
:1018430075E51D151D70DC151C80D8AF2D7E0012AB
:0D1853001D798006E522640160FA0220493B
:10141900121A64121FA4E537B40102C287122048C8
:101429009028CCE070067F8E7E0D80047FAA7E0511
:10143900121A1E121D9B122010121A99E539706A90
:10144900E52C75F040A485F01CF51DAF227E00AC9B
:101459001CAD1D1207FDD3EF9400EE940040147FDC
:10146900C47E03121D79121175E51D151D70DC1559
:101479001C80D8751C00852E1DAF227E00AC1CADCA
:101489001D1207FDD3EF9400EE940040147FC47E33
:1014990000121D79121175E51D151D70DC151C80D2
:1014A900D8AF2D7E00121D798006E522640160FA0D
:0A14B900122049E537B40102D28782
:0114C3002206
:0C1B1D00122010121A99C286AF3FAE3E93
:101B2900AD07AC06D3ED9400EC9400401E00000014
:101B3900EE90E6D0F0000000ED90E6D1F000000054
:0C1B490075BB04000000E5BB30E7FB2288
:081B55008C1C8D1DAB07AA06D4
:101B5D00E4FDFCC3ED951DEC951C5022EA90E6D0FA
:101B6D00F0000000EB90E6D1F000000075BB060020
:0E1B7D000000E5BB30E7FB0DBD00010C80D57C
:011B8B002237
:041CEC00AF26AE254C
:101CF000AD07AC06000000ED25E0EC3390E6D0F037
:101D0000000000ED25E090E6D1F000000075BB0476
:091D1000000000E5BB30E7FB22F6
:101DC500000000E53225E0E5313390E6D0F0000073
:101DD50000E53225E090E6D1F000000075BB040077
:081DE5000000E5BB30E7FB2222
:0812B8001215FBC206752201AC
:1012C0009028AEE0FFE4FCFDFEFB7A01F9F812087D
:1012D0000FC004C005C006C0079028ADE0FFE4FCC5
:1012E000FDFEFBFA7901F812080FD003D002D001FD
:1012F000D000EF2BFBEE3AFAED39F9EC38F89028F4
:10130000AFE0FFE4FCFDFEEB2FF53DEE3AF53CEDE2
:1013100039F53BEC38F53AE47F8EAB3DAA3CA93B6E
:10132000A83AD312092C401CE53D2471F53DE53C5B
:1013300034FFF53CE53B34FFF53BE53A34FFF53A45
:10134000C2088002D2082008101217D3E530452FBA
:101350007003121E9DD287800EE530452F70031258
:091360001E9D1217D3D287D2861C
:011369002261
:10136A009028AEE0FFE4FCFDFEFB7A01F9F81208D2
:10137A000FC004C005C006C0079028ADE0FFE4FC1A
:10138A00FDFEFBFA7901F812080FD003D002D00152
:10139A00D000EF2BFBEE3AFAED39F9EC38F8902849
:1013AA00AFE0FFE4FCFDFEEB2FF53DEE3AF53CED38
:1013BA0039F53BEC38F53A9028CCE0701E7F8E7EEA
:1013CA000DAB3DAA3CA93BA83AD312092C403CE5F7
:1013DA003D2472F53DE53C34F2801FE47FAA7E0588
:1013EA00FDFCAB3DAA3CA93BA83AD312092C401BF1
:1013FA00E53D2456F53DE53C34FAF53CE53B34FF42
:0F140A00F53BE53A34FFF53A020CFF120BDC22FA
:101860001212B8121F203006030218ECE4F518F526
:1018700019C3E5199529E5189528500D121E3C0548
:1018800019E51970EC051880E89028CCE070067D09
:101890000AFCFF80067D327C007F007E0D121B5506
:1018A000D3E5269400E52594004003121CECE4FDEA
:1018B000FCC3ED9546EC9545500A121E390DBD004E
:1018C000010C80EDE4F518F519C3E5199543E51809
:1018D0009542500D121E3C0519E51970EC05188053
:0C18E000E8122010121A99D286121B2563
:0118EC0022D9
:10156D001212B8121F203006030215FAE4F518F511
:10157D0019C3E5199529E51895285010121E3C122E
:10158D001E3C0519E51970E9051880E59028CCE099
:10159D0070067D0AFCFF80067D327C007F007E0D8B
:1015AD00121B55D3E5269400E52594004003121C2B
:1015BD00ECE4FDFCC3ED9546EC9545500D121E393E
:1015CD00121E3C0DBD00010C80EAE4F518F519C39F
:1015DD00E5199543E51895425010121E3C121E3C1C
:0D15ED000519E51970E9051880E5121B1DB0
:0115FA0022CE
:100CFF001215FBC206752201121419121E9D121D28
:100D0F00ED121F26300603020E1DE4F51AF51BC364
:100D1F00E51B9529E51A9528500D121E3C051BE57C
:100D2F001B70EC051A80E89028CCE070067D0AFC59
:100D3F00FF80067D327C007F007E0D121B55D3E5B0
:100D4F00269400E52594004003121CECE4F518F5F9
:100D5F0019E545C313FEE54613FFC3E5199FE518D3
:100D6F009E5010121DC5121E3C0519E51970E205A3
:100D7F001880DEE4F51AF51BC3E51B9543E51A95BC
:100D8F0042500D121E3C051BE51B70EC051A80E846
:100D9F00121D9BE4F51AF51BC3E51B9529E51A9562
:100DAF0028500D121E3C051BE51B70EC051A80E840
:100DBF009028CCE070067D0AFCFF80067D327C0017
:100DCF007F007E0D121B55E4F518F519E545C31389
:100DDF00FEE54613FFC3E5199FE5189E5010121D3F
:100DEF00C5121E3C0519E51970E2051880DEE4F501
:100DFF001AF51BC3E51B9543E51A9542500D121EBC
:0E0E0F003C051BE51B70EC051A80E8121B2346
:010E1D0022B2
:100BDC001212B8121DED121F26300603020CFEE491
:100BEC00F51AF51BC3E51B9529E51A9528500D122E
:100BFC001E3C051BE51B70EC051A80E89028CCE028
:100C0C0070067D0AFCFF80067D327C007F007E0D25
:100C1C00121B55D3E5269400E52594004003121CC5
:100C2C00ECE4F518F519E545C313FEE54613FFC3CF
:100C3C00E5199FE5189E5010121DC5121E3C051992
:100C4C00E51970E2051880DEE4F51AF51BC3E51B07
:100C5C009543E51A9542500D121E3C051BE51B7081
:100C6C00EC051A80E8122010121A991215FB1212B8
:100C7C00C0121D9B121F26E4F51AF51BC3E51B952C
:100C8C0029E51A9528500D121E3C051BE51B70EC2E
:100C9C00051A80E89028CCE070067D0AFCFF8006DF
:100CAC007D327C007F007E0D121B55E4F518F51982
:100CBC00E545C313FEE54613FFC3E5199FE5189EF2
:100CCC005010121DC5121E3C0519E51970E20518CD
:100CDC0080DEE4F51AF51BC3E51B9543E51A954236
:100CEC00500D121E3C051BE51B70EC051A80E8121A
:020CFC001B1DBE
:010CFE0022D3
:10093D001215FBC2067522019028AEE0FFE4FCFD06
:10094D00FEFB7A01F9F812080FC004C005C006C0FD
:10095D00079028ADE0FFE4FCFDFEFBFA7901F812EB
:10096D00080FD003D002D001D000EF2BFBEE3AFAE6
:10097D00ED39F9EC38F89028AFE0FFE4FCFDFEEB23
:10098D002FF53DEE3AF53CED39F53BEC38F53A12E5
:10099D0017D3121E9D121DED121F26300603020ADB
:1009AD00B2E4F51AF51BC3E51B9529E51A952850F8
:1009BD000D121E3C051BE51B70EC051A80E89028F6
:1009CD00CCE070067D0AFCFF80067D327C007F0046
:1009DD007E0D121B55D3E5269400E52594004003AA
:1009ED00121CECE4F518F519E545C313FEE54613A5
:1009FD00FFC3E5199FE5189E5010121DC5121E3C30
:100A0D000519E51970E2051880DEE4F51AF51BC32A
:100A1D00E51B9543E51A9542500D121E3C051BE54D
:100A2D001B70EC051A80E8121D9BE4F51AF51BC32B
:100A3D00E51B9529E51A9528500D121E3C051BE561
:100A4D001B70EC051A80E89028CCE070067D0AFC3E
:100A5D00FF80067D327C007F007E0D121B55E4F574
:100A6D0018F519E545C313FEE54613FFC3E5199FB8
:100A7D00E5189E5010121DC5121E3C0519E5197082
:100A8D00E2051880DEE4F51AF51BC3E51B9543E579
:100A9D001A9542500D121E3C051BE51B70EC051AF4
:050AAD0080E8121B238C
:010AB2002221
:081FAC00E4F562D2E9D2AF2294
:101BC20090E678E020E6F9C2E990E678E04480F019
:101BD200EF25E090E679F090E678E030E0F990E6E3
:101BE20078E04440F090E678E020E6F990E678E08C
:061BF20030E1D6D2E92229
:101C5E00A90790E678E020E6F9E562702390E67831
:101C6E00E04480F0E925E090E679F08D5DAF03A9C0
:101C7E0007755E018A5F8960E4F561756201D322A2
:021C8E00C3226F
:101BF800A90790E678E020E6F9E562702590E67896
:101C0800E04480F0E925E0440190E679F08D5DAF8D
:101C180003A907755E018A5F8960E4F5617562034F
:041C2800D322C322DE
:03004B00020E1E84
:100E1E00C0E0C083C082C085C084C086758600C015
:100E2E00D075D000C000C001C002C003C006C0070C
:100E3E0090E678E030E206756206020F0890E678DA
:100E4E00E020E10CE56264026006756207020F089D
:100E5E00E56224FE605F14603624FE7003020EF914
:100E6E0024FC7003020F0524086003020F08AB5E1A
:100E7E00AA5FA960AF6105618F827583001207AE0C
:100E8E0090E679F0E561655D7070756205806B9036
:100E9E00E679E0AB5EAA5FA960AE618E82758300D3
:100EAE001207DB756202E55D6401704E90E678E034
:100EBE004420F08045E55D24FEB5610790E678E0BC
:100ECE004420F0E55D14B5610A90E678E04440F008
:100EDE0075620090E679E0AB5EAA5FA960AE618EA6
:100EEE00827583001207DB0561800F90E678E0447F
:100EFE0040F075620080037562005391DFD007D019
:100F0E0006D003D002D001D000D0D0D086D084D06D
:080F1E0085D082D083D0E032BF
:030000000218EDF6
:0C18ED00787FE4F6D8FD758162021934A2
:1007AE00BB010CE58229F582E5833AF583E0225000
:1007BE0006E92582F8E622BBFE06E92582F8E2224A
:0D07CE00E58229F582E5833AF583E4932264
:1007DB00F8BB010DE58229F582E5833AF583E8F054
:1007EB00225006E92582C8F622BBFE05E92582C800
:0207FB00F222E8
:1007FD00EF8DF0A4A8F0CF8CF0A428CE8DF0A42E10
:02080D00FE22C9
:10080F00E88FF0A4CC8BF0A42CFCE98EF0A42CFC88
:10081F008AF0EDA42CFCEA8EF0A4CDA8F08BF0A406
:10082F002DCC3825F0FDE98FF0A42CCD35F0FCEB65
:10083F008EF0A4FEA9F0EB8FF0A4CFC5F02ECD392A
:0F084F00FEE43CFCEAA42DCE35F0FDE43CFC2297
:10085E0075F008758200EF2FFFEE33FECD33CDCC51
:10086E0033CCC58233C5829BED9AEC99E5829840D4
:10087E000CF582EE9BFEED9AFDEC99FC0FD5F0D6B1
:10088E00E4CEFBE4CDFAE4CCF9A88222B800C1B9DB
:10089E000059BA002DEC8BF084CFCECDFCE5F0CB19
:1008AE00F97818EF2FFFEE33FEED33FDEC33FCEB52
:1008BE0033FB10D703994004EB99FB0FD8E5E4F90D
:1008CE00FA227818EF2FFFEE33FEED33FDEC33FCFA
:1008DE00C933C910D7059BE99A4007EC9BFCE99AEE
:1008EE00F90FD8E0E4C9FAE4CCFB2275F010EF2F33
:1008FE00FFEE33FEED33FDCC33CCC833C810D70733
:10090E009BEC9AE899400AED9BFDEC9AFCE899F86D
:0E091E000FD5F0DAE4CDFBE4CCFAE4C8F92200
:10092C00EB9FF5F0EA9E42F0E99D42F0E89C45F021
:01093C002298
:1018F900020601E493A3F8E493A34003F68001F2FE
:1019090008DFF48029E493A3F85407240CC8C333EF
:10191900C4540F4420C8834004F456800146F6DFBE
:10192900E4800B0102040810204080900FF0E47E4F
:10193900019360BCA3FF543F30E509541FFEE493B3
:10194900A360010ECF54C025E060A840B8E493A37A
:10195900FAE493A3F8E493A3C8C582C8CAC583CAA5
:10196900F0A3C8C582C8CAC583CADFE9DEE780BE5D
:0110B8000037
:00000001FF
